:02000000BA281C
:08000800002882073334333471
:100010003234203406340C34013402342008820790
:100020000034013402340334043405340634073414
:10003000083409340A340B340C340D340E340F34C4
:100040008207A22B432C382DA72CCC2B612C6B2D97
:10005000D42CF32B792C882DF82C1A2C902CA32D32
:10006000182D8207282B5D2B822A872B8207533479
:100070007434613474346E34203423343134203495
:1000800020342334323420342034233433342034A5
:1000900020342334343400348207533465347234CA
:1000A000763469346334653420344D346F346434C9
:1000B000653420345034613467342F34523465341D
:1000C0006734003482072034203445346D3465347D
:1000D0007234673465346E34633479342034533485
:1000E00074346F347034213420342034203400349C
:1000F00082074D3469346E346934443443344334B4
:100100002034533474346134743469346F346E344D
:100110002034763435342E34373400348207543466
:10012000753472346E346F3475347434203443341F
:100130006F346E34743472346F346C3420344D3414
:100140006F346434653400348207463475346E3459
:100150006334743469346F346E34203443346F3410
:100160006E34743472346C3420344D346F346434EF
:1001700065340034DC20DE255B27D408031DCF283E
:100180006B27CE26D126D426D7266B27042708270F
:100190000C2710276418902256189022BD285B2740
:1001A0006B27D820D4080319C028D6189022D0284D
:1001B0006E26C1196426080007309F0083162C3074
:1001C0008500860183128601213084006030A00002
:1001D0008001840AA00BE82846308400B701370864
:1001E000D7258000840AB70A06303706031DEF289A
:1001F000FB229030CC00CD00CE00CF008030D70065
:10020000D900F830D800DA00DD0A4130E1000800FA
:10021000C1180800D408031D0800C1140430AE0042
:1002200056180800D40AD4305826B701370862207F
:10023000B70A003E03191E29402616294A08A800BD
:10024000CA010C234208EA004308EB004408EC0012
:100250004508ED004130C200C300C400C5006E1C5B
:10026000C216EE1CC3166E1DC416EE1DC5160A304E
:10027000A5001930B700E127851D57296B27CE2629
:10028000D126D426D7266B27A50B39292808CA00E2
:1002900056106A08C2006B08C3006C08C4006D08E1
:1002A000C5000C23F6251A26D401D4309B2BD4305C
:1002B0009B23C110D4012808CA005E29C118080078
:1002C000C1140430AE00FB225408D40A3128D619D8
:1002D00096296822D615EB25C0305826B701370875
:1002E000A420B70A003E0319772940266F29F82574
:1002F000D430582659275927592759274C3084007C
:100300000430BA002D3000182A3040262D308018D5
:100310002A3040262D3000192A3040262D308019F1
:100320002A304026840ABA0B82290800D601D4015B
:10033000DE2DDF0ADF0ADF0ADF0ADF0ADF0ADF0A53
:10034000DF0ADF0A6008DB00DC00DB0DDB0DDB0D04
:100350005C0D5B075F07CB0058105A105F08E00088
:10036000DF01080094305826523040266530402680
:10037000633040262E304026CB29561C0800D61963
:10038000080094305826503040266C3040266130AA
:100390004026793040265927523040266F3040267B
:1003A0007530402674304026653040265927610854
:1003B000402659275D084E2659274B087F394E267F
:1003C0007C30CB1B2F304026192A56190800DD0A35
:1003D00004305D076707D725A90803195615CB0018
:1003E00008005611DD0BE829DD0A080061085A3AB9
:1003F00003190800E10A022A6108413A03190800BA
:10040000E103022A5611E701413061020319122A61
:10041000E80005306707D725E70AA908031D092A60
:10042000E80B092A0130DD0005306707D725CB002E
:1004300008007B30E900B4000530B2003208D7254F
:10044000A908031DE903B20AB40B1E2AD4305826AA
:100450005B304026690852265D30402ECB080319D8
:10046000412A5818CB1704305D076707EA00D725E3
:10047000A90803194A224B08A2006A08BE25561192
:10048000E52904305D076707EA00D725A908031DA1
:10049000592208006A08803CEB008030E5006508BE
:1004A000E5036508D725A200650ABE25EB0B502A97
:1004B00008006A08803CEB006A08E5006508E50A68
:1004C0006508D725A2006503BE25EB0B5F2AE82946
:1004D000B501013040265C2EC1180800C11404305B
:1004E000AE00561C742A672968225614EB25C030CA
:1004F0005826B70137088E20B70A003E0319BD29D8
:1005000040267A2A6822D614EB25C0305826B70137
:1005100037088E20B70A003E0319B2294026882AE0
:100520006418AE2A59085702031D992A5A0858021E
:10053000031D9D22D61CBD29B2295708D900580891
:10054000DA007D275708BD00B9008A27B12758086F
:10055000BE00B9008A27BF01C001972FE608031D1E
:10056000B52A05306707E500DD01E60A6608323A7C
:10057000031D0800E601E60A6508D725E50AA90873
:100580000319CC2ADD0AC42ACB00A91FCA2AF822E3
:100590006B27992AD222C82A6410E601DD080319C4
:1005A000DD0A08005810CB134B08033EDB00D701CF
:1005B000D717D81058110310DB0C0318D8140310E8
:1005C000DB0C031858150310DB0C03185714031029
:1005D000DB0C0318D7140310DB0C0318571503109A
:1005E000DB0C0318D7150310DB0C03185716080093
:1005F0005814CB17D42A60304A1A8030C2006030B9
:10060000CA1A8030C30060304A1B8030C40060309A
:10061000CA1B8030C500EE01E030C205C305C40529
:10062000C5054A1C4216CA1C43164A1D4416CA1D5B
:10063000451680304A1AC205CA1AC3054A1BC405AA
:10064000CA1BC505D001D101D201D301AD010800FB
:10065000C0305826B70137083620B70A003E0319C4
:10066000332B40262B2B94305826413040266430C3
:100670004026643040267230402620304A1C3C30F0
:100680004A1A3E304026460852262030CA1C3C30CA
:10069000CA1A3E3040264708522620304A1D3C30B8
:1006A0004A1B3E304026480852262030CA1D3C30A6
:1006B000CA1B3E3040264908522EC0305826B7018A
:1006C00037084C20B70A003E0319682B4026602BE0
:1006D000D20A9430582643304026563040263A30CD
:1006E00040262D08AC005008013E522620304026FE
:1006F00056304026613040263A3040265108522676
:100700005927520852262D30402653084E2EFB22E0
:10071000D401B701D601463084000008A200370892
:10072000BE25840AB70A05303706031D8D2B6822C3
:10073000F6251A26EB2D58261430D5005927D50B4F
:100740009E2B0800D619C92B5618C52BD618C82BB6
:10075000D408031DB22B10304A1AB02B4A1CC20613
:10076000CC060800D4180800541C08004C164A187F
:10077000BD2B4A1ABF2B4A16332B4A10C12B4A12E3
:100780004A1442124A1C4216332B6414E601080034
:100790002E2A0830CC067829D619F02B5618EF2BC4
:1007A000D618EF2BD408031DDC2B1030CA1ADA2B15
:1007B000CA1CC306CD060800D4180800541C080043
:1007C0004D16CA18E72BCA1AE92BCA16332BCA10C2
:1007D000EB2BCA12CA144312CA1C4316332BFC2932
:1007E0000830CD067829D619172C5618162CD6188D
:1007F000162CD408031D032C10304A1B012C4A1D53
:10080000C406CE060800D4180800541C08004E1672
:100810004A190E2C4A1B102C4A17332B4A11122C42
:100820004A134A1544124A1D4416332BF629083040
:10083000CE067829D619402C56183D2CD6183D2CBA
:10084000D408031D2A2C1030CA1B282CCA1DC5062B
:10085000CF060800D4180800541C08004F16CA1907
:10086000352CCA1B372CCA17332BCA11392CCA1383
:10087000CA154512CA1D4516332B5818D22AF82A14
:100880000830CF067829D6195E2C56185D2CD6185C
:100890005D2CD418522C20304A1A8030C206013008
:1008A000EE0608005B275208B10014275B272627B5
:1008B0005B270130B10014275B2FF1290430CC06EF
:1008C0007829D619762C5618752CD618752CD4186C
:1008D000702C2030CA1A8030C3060230EE060800A1
:1008E0005B275008D30026275B2F99290430CD06BB
:1008F0007829D6198D2C56188C2CD6188C2CD418F7
:10090000882C20304A1B8030C4060430EE060800D4
:100910005B27502750275B2F9C290430CE0678296F
:10092000D619A42C5618A32CD618A32CD4189F2C57
:100930002030CA1B8030C5060830EE0608005B2751
:10094000382738275B2F9F290430CF067829D619FE
:10095000D12C5618D02CD618D02C5418C12CD41801
:10096000C42C1F304A1C0F304A1A7F30500603191E
:100970000800D00A4A1CBF2C1030C206421EC20A10
:100980000800C60A33230800D00AFF3050060319B6
:10099000AD0AD30A5319CD2C692BD301D20A692B86
:1009A000E5290130CC067829D619F52C5618F42CF7
:1009B000D618F42C5418EE2CD418F12C1F30CA1C65
:1009C0000F30CA1A7F30510603190800D10ACA1C19
:1009D000EC2C1030C306431EC30A0800C70A332399
:1009E0000800D10A692B08009B290130CD0678291F
:1009F000D619152D5618142DD618142D5418122D3D
:100A0000D41808001F304A1D0F304A1B7F30520691
:100A100003190800D20A4A1D102D1030C406441EC6
:100A2000C40A0800C80A332B9E290130CE06782953
:100A3000D619352D5618342DD618342D5418322D7C
:100A4000D41808001F30CA1D0F30CA1B7F30530650
:100A500003190800D30ACA1D302D1030C506451EE3
:100A6000C50A0800C90A332BA1290130CF0678290D
:100A7000D619682D5618672DD618672D54184D2D88
:100A8000D418502D500803190800D0034A1C4B2DD0
:100A90001030C206421AC2030800C60333230800FE
:100AA000D30353195D25D003FE3050060319AD035F
:100AB000FF302D0603196125692B0330D300D203C3
:100AC00008000230AD07D3008030D2000800A22910
:100AD0000230CC067829D619852D5618842DD618C3
:100AE000842D5418802DD418822D51080319080024
:100AF000D103CA1C7E2D1030C306431AC30308005D
:100B0000C703332BD103692B9A290230CD067829EC
:100B1000D619A02D56189F2DD6189F2D54189D2DEF
:100B2000D4180800520803190800D2034A1D9B2D4F
:100B30001030C406441AC4030800C803332B9D298F
:100B40000230CE067829D619BB2D5618BA2DD618E4
:100B5000BA2D5418B82DD4180800530803190800EA
:100B6000D3031030CA1DB62DC506451AC5030800AB
:100B7000C903332BA0290230CF067829A600D72538
:100B8000220603190800260883169B001C158B13E8
:100B90008312220883169A0055309D00AA309D00CA
:100BA0009C149C18D12D1C118B17831208008316DE
:100BB0009B001C141A088312A90008005C26B701C8
:100BC000B501370805204026B70AB71DE12D5C2680
:100BD000EB25F6251A2E80305826B70137087820E5
:100BE000B70A003E031908004026EE2DC030F92D4B
:100BF000943058264C3040266F30402663304026D3
:100C00003A304026460852262D304C1A2A304026CB
:100C1000470852262D304D1A2A30402648085226C1
:100C20002D304E1A2A304026490852262D304F1AB0
:100C30002A30402E943058265927592759275927AA
:100C40007E306E187F304026500852267E30EE18D7
:100C50007F304026510852267E306E197F30402664
:100C6000520852267E30EE197F3040265308522E0D
:100C7000B400340E0F393038402634080F3930387C
:100C8000B2002830A300A30B432E4626B20E320832
:100C90000F3935048600851485100800BC00C02774
:100CA0002A08382EBC00C02728083E262A08382EDD
:100CB00035124026351608002830A3009630B700BC
:100CC000E927A30B5E2E08002F082020C111D408AD
:100CD000031D080056180800F6251A2E051D762E4D
:100CE00085197A2ED408031D5E296C2AD408031DA9
:100CF0005E290829C11C842EAE0B0800C1103230B9
:100D0000AE000C30E2000800BD26EF30A40006085B
:100D10000B10A40C031CA62E2408860000000B1C3C
:100D2000872E41189D2E4114060EA700A826AF005D
:100D3000C1140430AE00C115C72EAE0BC72E0C3047
:100D40006202031DE2036208AE009B2E41109C2E3E
:100D5000A001A41DB22EA00A241DB22EA00AA41C1C
:100D6000B22EA00A271C0E28A71CBB2E271DB92EA9
:100D70002015A0150E2820150E280608B600FF30F5
:100D8000860083168113F03086008312080036082F
:100D90008600831681178601831208007D27DA26D4
:100DA000E52E7D27DC26E92E7D27DE26ED2E7D270C
:100DB000E026F12E4608E12E4708E12E4808E12EF4
:100DC0004908BD00B9008A27B12F42084A1AFA2EF5
:100DD000F42E4308CA1AFA2EF42E44084A1BFA2E9F
:100DE000F42E4508CA1BFA2EBE00B9008A27BF019F
:100DF000C001972FBF003F30BE00B9008A27B1273E
:100E00003F08B9008A27F82E7D27DA264C08F42EF1
:100E10007D27DC264D08F42E7D27DE264E08F42E95
:100E20007D27E0264F08F42E0630B3007B277D3067
:100E3000B900BD008A27B1273108BE00B9008A2752
:100E4000BF01C0019727B30B162F08000630B3006F
:100E50007B2753087F397838B900BD008A27B1272E
:100E60005108BE00B9008A279727B30B282F080026
:100E70007D27B901BD018A27B127EC30BE002D18AE
:100E80003E14AD18BE14B9008A27B1275008BF0020
:100E9000B9008A27B1275108C000B9008A27972FC7
:100EA0007B27BE017C30BD002D183D14AD18BD144C
:100EB000432F2030402E1430B2007D27B901BD01F0
:100EC000BE018A27B127B9018A27BF01C001972730
:100ED000B20B5D2F08007D27FF30B900BD008A27C7
:100EE000712F722F732F0000B127B901BE018A271D
:100EF000BF01C001972F19307E2F0F30A300802F24
:100F0000812F0000A627A30B7F2F862F872F882FE6
:100F10000000B12F0830BB000310B91F952FA62782
:100F2000912FB90DBB0B8D2F0800B127912FB12741
:100F30003D083E063F064006B9008A27A627BF01A6
:100F4000C001D4080319D820B12F0800A72F0330FF
:100F5000B700E927BD27AC2F00000430B700E92710
:100F6000BD2FB22F00000730B700E927BD2708309A
:100F7000B92FBA2FB700E927BD2F01308506080029
:100F800003101030BA00A501A801AA01BC0DAC0DD8
:100F9000AA0DA80DA50DBA0BCE2F00342A30D527E7
:100FA0002830D5272530D527C62F840003300007E9
:100FB000A100A119800030300007A100A11B800012
:100FC00000343708D500C8303708E927D50BE32FA0
:100FD00000340000EB2FEC2F0130B8000000F02FA0
:0A0FE000B80BEE2FB70BEC2F003416
:02400E00303F41
:1042000003000400050006000F000000000000008D
:10421000000000000000000000000000000000009E
:10422000000000000000000000000000000000008E
:10423000000000000000000000000000000000007E
:10424000000000000000000000000000000000006E
:10425000000000000000000000000000000000005E
:10426000000000000000000000000000000000004E
:10427000000000000000000000000000000000003E
:10428000000000000000000000000000000000002E
:10429000000000000000000000000000000000001E
:1042A000000000000000000000000000000000000E
:1042B00000000000000000000000000000000000FE
:1042C00000000000000000000000000000000000EE
:1042D00000000000000000000000000000000000DE
:1042E00000000000000000000000000000000000CE
:1042F00000000000000000000000000000000000BE
:00000001FF
